:10000000672CFF3FFF3FFF3F063003138312FA00C8
:10001000FA0B08280000080003138312200884004C
:100020000008F0002108F004200884007008800017
:100030000420200884000008F0002208F0052008B1
:100040008400700880000800031383122230FC0033
:10005000F801F901FA01FB01FC0303195A28031006
:10006000FB0CFA0CF90CF80CF30CF20CF10CF00C84
:10007000031C2C28FC0303194C287408F807750886
:100080000318750FF90776080318760FFA07770833
:100090000318770FFB0730287408F8077508031852
:1000A000750FF90776080318760FFA077708031813
:1000B000770FFB0708007C34A23492348A347C34F6
:1000C00000348434FE34803400348434C234A234A6
:1000D00092348C34423482348A34963462343034EC
:1000E00028342434FE3420344E348A348A348A341A
:1000F0007234783494349234923460340234E2347A
:1001000012340A3406346C349234923492346C349F
:100110000C349234923452343C3400340034003481
:100120000034003440342034103408340434FE34B5
:10013000FE347C3438341034003400340434003459
:10014000003400340034053400340034003400340A
:1001500006340034003400340034073400340034F2
:10016000FC34223422342234FC34FE34923492346F
:1001700092346C347C348234823482344434FE349D
:100180008234823444343834FE349234923492349B
:100190008234FE3412341234123402347C34823409
:1001A00082349234F434FE34103410341034FE347B
:1001B00000348234FE34823400344034803482345B
:1001C0007E340234FE341034283444348234FE3415
:1001D0008034803480348034FE3404341834043461
:1001E000FE34FE34083410342034FE347C3482343F
:1001F000823482347C34FE341234123412340C349F
:100200007C348234A2344234BC34FE34123432346E
:1002100052348C348C3492349234923462340234BA
:100220000234FE34023402347E348034803480342C
:100230007E343E344034803440343E347E34803426
:10024000703480347E34C634283410342834C634B4
:100250000E341034E03410340E34C234A2349234EC
:100260008A348634080003138312200884000008AF
:10027000F0002308F0052408F00520088400700829
:100280008000B8304804F000250884007008800021
:100290000C20080003138312200884000008F000DB
:1002A0002208F005200884007008800020088400DF
:1002B0000008F0002608F004200884007008800080
:1002C000200884000008F0002408F00520088400BD
:1002D0007008800025088400480880000C20080071
:1002E000031383124808A7004908A800A901AA011E
:1002F0000130AB00080003138312FD01F31F8D29A9
:10030000F009F109F209F309F00A0319F10A0319D6
:10031000F20A0319F30A8130FD07F71F9B29F4093C
:10032000F509F609F709F40A0319F50A0319F60A9B
:100330000319F70AFD0A24207D1CB529F009F109EB
:10034000F209F309F809F909FA09FB09F00A031996
:10035000F10A0319F20A0319F30A0319F80A031937
:10036000F90A0319FA0A0319FB0A08007F3003137C
:1003700083124805F1007108C800711FD4292008B4
:1003800084000008F0002C08F004200884007008A5
:100390008000200884000008F0002D08F0052008E7
:1003A000840070088000E829200884000008F0001C
:1003B0002E08F005200884007008800020088400C2
:1003C0000008F0002F08F004200884007008800066
:1003D00008007F3003138312C8052008840000083A
:1003E000F0002308F0052008840070088000200831
:1003F00084000008F0002408F0052008840070083C
:100400008000BF304805F0007008C8007017700801
:10041000C80025088400700880000C200800031321
:100420008312200884000008F0002608F004200849
:10043000840070088000200884000008F000220872
:10044000F00520088400700880002008840000085F
:10045000F0003008F004200884007008800080302C
:100460002507F1007108B100710884000008F00050
:100470003208F004710884007008800020088400AD
:100480000008F0002108F0042008840070088000B3
:10049000250884000008C800200884000008F00037
:1004A0002208F005200884007008800020088400DD
:1004B0000008F0002408F00520088400700880007F
:1004C000310884000008F0003308F005310884008A
:1004D000700880004808F0000800031383124708E2
:1004E000A5004008A000B301FF30B2004108F100B0
:1004F0000130F00071080319812AF00D7010FF3FE0
:100500007B2A7008AC007009AE004208F10001308F
:10051000F00071080319902AF00D7010FF3F8A2A2D
:100520007008AF007009AD004308F1000130F00021
:10053000710803199F2AF00D7010FF3F992A700867
:10054000A6007009A3004408F1000130F000710812
:100550000319AE2AF00D7010FF3FA82A7008B000F2
:100560007009A4004508F1000130F000710803197A
:10057000BD2AF00D7010FF3FB72A7008B400700953
:10058000B5004608F1000130F00071080319CC2ACB
:10059000F00D7010FF3FC62A7008A1007009A2007C
:1005A00080304707F1007108B1007108840000082D
:1005B000F0000030F0057108840070088000803081
:1005C0002007F1007108B100710884000008F000F4
:1005D0002E08F0057108840070088000310884003E
:1005E0000008F0002D08F005310884007008800034
:1005F000310884000008F0002308F0053108840069
:1006000070088000310884000008F0002408F0051C
:100610003108840070088000310884000008F00070
:100620003508F00531088400700880003108840026
:100630000008F0002208F0053108840070088000EE
:10064000200884000008F0003408F004200884002A
:1006500070088000200884000008F0002308F005DE
:100660002008840070088000200884000008F00042
:100670002408F00520088400700880002008840009
:100680000008F0002E08F0052008840070088000A3
:10069000200884000008F0002F08F00420088400DF
:1006A00070088000250884003F3080000C20250859
:1006B0008400C03080000C20200884000008F00076
:1006C0002C08F004200884007008800020088400B2
:1006D0000008F0002D08F005200884007008800054
:1006E000250884003F3080000C2025088400C0309D
:1006F00080000C200530B6000730B7005B30B80032
:100700000030B9003030BA000030BB0008000313DD
:100710008312200884000008F0002E08F0052F083E
:10072000F0042008840070088000C2014208073CE1
:10073000031CA92B4208C8003321C10141083F3CDA
:10074000031CA72B4008C8004A21C10A9E2BC20ADD
:10075000962B200884000008F0002D08F0052C08D6
:10076000F0042008840070088000C2014208073CA1
:10077000031CC92B4208C8003321C10141083F3C7A
:10078000031CC72B4008C8004A21C10ABE2BC20A5D
:10079000B62B0800031383122B08031DD42B013042
:1007A000C8000030C90070212708F0002808F100B7
:1007B0002908F2002A08F3006D30F4004E30F500ED
:1007C000C630F6004130F7007B213930F50030307B
:1007D000F600F701F8017008F50771080318710FAA
:1007E000F60772080318720FF70773080318730FE0
:1007F000F8077708F0007808F100F201F301FF3004
:10080000F0057F30F1050030F205F3057008A70010
:100810007108A8007208A9007308AA0008007F30B8
:10082000031383124005F0007008C0003F30C1057B
:100830007008C800B6214108C800C80CC813C80C0D
:10084000C813C80CC81333214008C800E9210F227F
:100850007008C4000F227008C4004108C800C80C0A
:10086000C813C80CC813C80CC81333214008C800EB
:10087000E92107304105F0007008C3007008F1005D
:100880000130F00071080319492CF00D7010FF3F82
:10089000432C7008C3007009C500572C4508C405D7
:1008A000632C4308C404632C4308C406632C420829
:1008B000003A03194E2C4208013A0319512C420800
:1008C000023A0319542C4408C8004A2108000313B3
:1008D00083168701913083128700831686016E305C
:1008E000831286000630C000C1010130C200023010
:1008F000C3000330C4000530C5000430C600083012
:10090000C7006D22C001872380303D06F000803093
:10091000013A7002031D8E2C00303C020318952C06
:10092000CA23BC0A0319BD0A842CCA237008BE005E
:100930007108BF00CA237008C0000230C2003E0820
:10094000C1000F24952CA32CFF3FFF3FFF3FFF3F2B
:02400E007A3FF7
:00000001FF
